:100000000C9441000C945E000C945E000C945E0015
:100010000C945E000C945E000C945E000C945E00E8
:100020000C945E000C945E000C945E000C94C00274
:100030000C945E000C945E000C945E000C945E00C8
:100040000C945E000C945E000C94B5000C945E0061
:100050000C945E000C9460000C945E000C945E00A6
:100060000C945E000C945E00244750524D430024D3
:100070004750474741002E6C6F6700244750524D50
:10008000430011241FBECFEFD4E0DEBFCDBF11E08F
:10009000A0E0B1E0EAEAF3E202C005900D92A630DA
:1000A000B107D9F714E0A6E0B1E001C01D92AF336B
:1000B000B107E1F70E9435010C94D3110C940000B4
:1000C0001F920F920FB60F9211242F933F938F938D
:1000D000209178003091790080917C00203D31059D
:1000E00070F4809109018F3030F08091650181605A
:1000F0008093650106C08F5F8093090102C0109252
:10010000090181E02C32380770F0809108018F30AE
:1001100030F0809165018E7F8093650106C08F5F0E
:100120008093080102C01092080130936701209368
:10013000660182E480937C0080917C00309302020F
:100140002093010281E480937C008FED80937A00FC
:100150008F913F912F910F900FBE0F901F90189588
:1001600060E070E081EA96E308951F920F920FB667
:100170000F9211248F939F93EF93FF939091C6005A
:1001800080916A01863988F48F5F80936A0180913B
:100190006801E82FF0E0E859FE4F93838F5F8639BE
:1001A00008F080E08093680105C08091650182605D
:1001B00080936501FF91EF919F918F910F900FBEFA
:1001C0000F901F90189590E051E448E901C090E02D
:1001D0008091650180FD46C03091690180916A017E
:1001E000882311F420E013C0E32FF0E0E859FE4F1C
:1001F0002381E32FEF5FF89480916A01815080930F
:100200006A017894E63908F0E0E0E09369018091B2
:10021000650181FF14C0F8941092C1001092690129
:100220001092680110926A015093C4004093C1007B
:10023000809165018D7F809365017894C8CF2223DA
:1002400039F2992319F4243209F0C2CFE92FF0E0F2
:10025000ED5EFE4F20839F5F2A3029F0923508F033
:10026000B6CFB6CF90E0892F0895A2E0B0E0EBE3DF
:10027000F1E00C94A1118DE085B98EE284B98FE391
:1002800088B917B88EEA8BB982E58AB980E58CBD4A
:1002900081E08DBD83ED90E3909389008093880089
:1002A0008AE08093810082E080936F0082E187BDC5
:1002B00082E484BD81E480937C008FED80937A009A
:1002C00078946FE172E080E00E942709EE24FF2419
:1002D00034E6832E77247A9423E0C22E95E0D92E3B
:1002E0005E010894A11CB11C82E3982E1092C100FB
:1002F0002998809212018091650180FF02C080924E
:100300001201809112018823B1F7299A709212018B
:100310008091650180FD05C080E00E943D0F81FF56
:1003200002C07092120180911201882389F791E036
:100330000EC0C5BCD0921201809112018823E1F752
:1003400015BCD0921201809112018823E1F79150DF
:1003500080F7F8941092C100109269011092680120
:1003600010926A0181E48093C40088E98093C100FF
:10037000809165018D7F80936501789402C0EE24A1
:10038000FF240E94E300882309F4B0CF2BE730E07C
:10039000A3E1B1E0F9012F5F3F4F9491992329F038
:1003A0008C91981771F41196F5CFE3E1F1E082E0BA
:1003B0009081913220F331969C32D1F78150C1F770
:1003C0007F01E114F104E9F2F70180818134C9F67B
:1003D000E3E1F1E089E09081913208F4A6C0319622
:1003E0009C32C9F78150B9F77F01309709F49DC05D
:1003F000848195819093140180931301828193816C
:10040000909316018093150180819181909318013A
:100410008093170166E770E089E191E00E9437114F
:1004200042E163E171E083E092E00E947F09892B61
:1004300009F07DC040910D0250910E0260910F02B3
:100440007091100283E092E00E94E404892B09F08D
:100450006EC092E00EC0C5BCD09212018091120114
:100460008823E1F715BCD0921201809112018823F4
:10047000E1F7915080F73FC02FE630E0A3E1B1E013
:10048000F9012F5F3F4F9491992389F08C91981730
:1004900009F064C01196F4CF1196F9012F5F3F4F18
:1004A0009491992321F08C919817B1F311C0042FE6
:1004B00010E09501A80163E171E083E092E00E9401
:1004C000B606892BF9F489819A8108171907D1F4A6
:1004D0008091650182FF0FC083E092E00E94510687
:1004E000892B11F096E024C0F894809165018B7FF0
:1004F0008093650178940E94E300482F882309F0D7
:10050000BBCF31C095E014C0C5BC90921201809160
:1005100012018823E1F715BC90921201809112011B
:100520008823E1F7915080F7E1CE93E001C094E099
:100530001092C100299833E029E135BD20931201C2
:10054000809112018823E1F715BC2093120180915C
:1005500012018823E1F7915081F7FFCF28E630E0C0
:10056000A3E1B1E09ACF1092C100299883E092E014
:100570000E94A806892B11F097E0DACF91E0D2CF44
:100580001F920F920FB60F9211242F938F939F9368
:1005900080911201882319F081508093120180917B
:1005A000060190910701019690930701809306013F
:1005B0008055964448F010920701109206018091F0
:1005C00065018460809365010E9417119F918F914E
:1005D0002F910F900FBE0F901F901895FC01009760
:1005E00069F0808191818617970741F480E00E942D
:1005F0003D0F282F30E02170307002C02CE030E039
:10060000C9010895A0E0B0E0E8E0F3E00C94A01187
:100610004B015C01C0910A01D0910B01CC80DD80BF
:10062000EE80FF80C616D706E806F90609F44EC02C
:100630008F8D8823A1F180E2682E712C6C0E7D1EB7
:1006400001E0A7019601B30180E00E94A30F892B6E
:10065000D9F51F8E8C899D89A0E0B0E02885398569
:100660004A855B85820F931FA41FB51FC816D90644
:10067000EA06FB06A0F41E8D10C08C899D89A0E0BF
:10068000B0E0C80ED91EEA1EFB1E01E0A7019601CC
:10069000B30180E00E94A30F1150123070F7811453
:1006A0009104A104B10491F0BE01605E7F4F01E0AE
:1006B000A501940180E00E94440F892B29F48C82CB
:1006C0009D82AE82BF8202C080E001C081E0CDB7D2
:1006D000DEB7EEE00C94BC11A0E0B0E0E2E7F3E09E
:1006E0000C94A011EC014B01E0900A01F0900B0179
:1006F000F701A084B184C284D384848D813021F039
:10070000823009F072C05AC08E01000F111F0C0F09
:100710001D1F16950795B801672F7727669580E00E
:1007200090E06A0D7B1D8C1D9D1D0E940203882395
:1007300009F45BC0D801B17051E0652E712C6C22B8
:100740007D22C0FF0AC0F701EA0FFB1F80A18F7056
:10075000982D9295907F982B01C0982DAE0DBF1DBE
:10076000FD0190A3E801219681E0F701878FBE018A
:10077000672F7727669580E090E06A0D7B1D8C1DC2
:100780009D1D0E940203882381F1DE01B170611476
:10079000710439F034E0969487943A95E1F7982DF6
:1007A00008C0F701EA0FFB1F90A1907F892D8F7081
:1007B000982BAE0DBF1DFD0190A313C06D2F7727A1
:1007C00080E090E06A0D7B1D8C1D9D1D0E94020340
:1007D000882359F0CC0FDD1FD170CE0DDF1D99A2FB
:1007E00088A281E0F701878F01C080E0CDB7DEB736
:1007F000EEE00C94BC11A0E0B0E0E1E0F4E00C9479
:10080000A3118C01E0900A01F0900B018230910558
:1008100008F467C0E7018E899F890817190708F057
:1008200060C0A884B984CA84DB848C8D813021F0B7
:10083000823009F056C040C0E801CC0FDD1FC00F68
:10084000D11FD695C795BE01672F7727669580E0A3
:1008500090E06A0D7B1D8C1D9D1D0E940203882364
:1008600009F43FC0FE01F170EE0DFF1D90A021962E
:10087000BE01672F7727669580E090E06A0D7B1DAB
:100880008C1D9D1D0E940203882359F1292D30E003
:10089000D170EC0EFD1EF70190A180E0282B392BC2
:1008A00000FF07C0F90194E0F695E7959A95E1F706
:1008B0001AC0F901FF7017C0612F772780E090E020
:1008C0006A0D7B1D8C1D9D1D0E940203882349F02B
:1008D000000F111F1170E00EF11EE701E8A1F9A150
:1008E00002C0E1E0F0E0CF01CDB7DEB7EBE00C9461
:1008F000BF11A0E0B0E0EFE7F4E00C94A4117C019C
:10090000C0900A01D0900B01F601A688B788009725
:1009100049F4008D118D0230110588F00A151B0570
:1009200070F40FC00E94FB039C018230910508F413
:1009300040C08A159B0508F441C0870102C001E050
:1009400010E0E8012196CA15DB0528F002301105F8
:1009500098F1C2E0D0E0CE010E94FB039C01009719
:1009600039F08130910551F1C017D10759F724C0F2
:100970001C2F0D2F6FEF7FEFCE010E946C03882399
:10098000C1F0E114F10431F0BE01C7010E946C0313
:10099000882379F0F601108F018F828D938DFFEF00
:1009A0008F3F9F0721F00197F601938F828F9E0161
:1009B00005C021E030E002C020E030E0C901CDB741
:1009C000DEB7EAE00C94C011A0E0B0E0EAEEF4E09B
:1009D0000C94A011EC017A018B016C807D80688100
:1009E0007981C3010E94EE024C01009709F0D6C044
:1009F0008A8187FDD0C0AA84BB84CC84DD84AE14F8
:100A0000BF04C006D10610F481FF02C0570168017F
:100A10001E821F821886198681E08B83A114B1047F
:100A2000C104D10409F49DC06E857F8561157105EF
:100A300071F480E090E00E947904BC01813091055E
:100A400009F4A6C09F878E87009709F48AC0F30136
:100A5000858DE82EFF2400E010E0F9E0EE0CFF1C8D
:100A6000001F111FFA95D1F7798B688BEA14FB04EC
:100A70000C051D0558F58A8181FF04C0CB010E9439
:100A8000790403C0CB010E94FB03BC010097E1F095
:100A90008130910509F47CC0F30186899789681734
:100AA000790708F075C08E819F81A885B9858E0D64
:100AB0009F1DA01FB11F8E839F83A887B987AE1883
:100AC000BF08C00AD10AD0CF57016801D601C501BD
:100AD0000197A109B109E9E0B695A7959795879582
:100AE000EA95D1F7F82E00910A0110910B0162509E
:100AF0007040F8018689978902976817790728F06E
:100B000020E030E040E050E014C080E090E0F801E8
:100B1000258D30E040E050E00E945B119B01AC016C
:100B2000F80180899189A289B389280F391F4A1F4A
:100B30005B1F2F0D311D411D511D2A8B3B8B4C8B93
:100B40005D8BF301858D8F198B838E819F81A885A5
:100B5000B9858A0D9B1DAC1DBD1D8E839F83A88703
:100B6000B9876A8161FF1AC02E813F814885598506
:100B70008A859B85AC85BD8582179307A407B50739
:100B800068F42A873B874C875D8760626A8306C06A
:100B90008A8180688A8368E0862E912CC401CDB753
:100BA000DEB7EEE00C94BC11EF92FF920F931F930F
:100BB000CF93DF938C01C0910A01D0910B01FC010E
:100BC000E280F3800894E11CF11CC7018F709070E3
:100BD000892B09F05BC082859385A485B585019634
:100BE000A11DB11D82879387A487B5874085518554
:100BF0004115510539F48A819B81E816F90608F4FC
:100C000045C049C08D8D90E001979701A4E03695CD
:100C10002795AA95E1F782239323892BB9F5CA0179
:100C20000E94FB03BC0182309105A8F18E899F8947
:100C30006817790780F5F80171876087C0910A010C
:100C4000D0910B01625070408E899F89029768177E
:100C5000790728F020E030E040E050E012C080E06A
:100C600090E02D8D30E040E050E00E945B119B0150
:100C7000AC0188899989AA89BB89280F391F4A1F25
:100C80005B1FF8012287338744875587F801F38279
:100C9000E28281E001C080E0CDB7DEB7E6E00C94EF
:100CA000C411EF92FF920F931F93CF93DF93EC0148
:100CB000688179818C819D810E94EE027C01009780
:100CC00009F040C08A8185FF3DC06E897F89888D8B
:100CD000998D0E940203882391F10A8D1B8DF801E2
:100CE0008385806283878A859B85AC85BD85848F5B
:100CF000958FA68FB78F8E859F85938F828F0E9449
:100D0000B000F801668B778B808F918F8A818F7D01
:100D10008A83E0910A01F0910B0181E0878F60E006
:100D200070E080E090E00E940203882341F040E000
:100D300050E063E080E00E941F10892B19F0B8E0BA
:100D4000EB2EF12CC701CDB7DEB7E6E00C94C41151
:100D5000CF93DF93EC010E9451069C01009711F4A0
:100D60001D821C82C901DF91CF910895A0E0B0E0FF
:100D7000ECEBF6E00C949D11EC01162F072F7A0195
:100D80003901AC80BD80F9011182108268817981BE
:100D9000C5010E94EE024C01009709F03BC18A8117
:100DA00087FD35C181FD04C036E0832E912C32C110
:100DB0002A853B854C855D85C701A0E0B0E0820FA8
:100DC000931FA41FB51F82179307A407B50708F444
:100DD00021C1812F902F9C016901412C22E0522ECC
:100DE00033243394F8C02E813F8148855985DA0138
:100DF000C9019170A070B0700097A105B10509F00C
:100E0000B1C08B8181508B83882349F02A893B892B
:100E10004C895D892F5F3F4F4F4F5F4F51C0211568
:100E200031054105510569F46E857F8561157105B0
:100E300089F480E090E00E947904BC019F878E874E
:100E400005C0888999890E947904BC0161157105E2
:100E500009F4C5C06130710509F4D6C0F501868971
:100E600097896817790708F0CFC0798B688B009154
:100E70000A0110910B0162507040F8018689978930
:100E800002976817790728F020E030E040E050E052
:100E900014C080E090E0F801258D30E040E050E0A3
:100EA0000E945B119B01AC01F80180899189A289A4
:100EB000B389280F391F4A1F5B1FF501858D8B836E
:100EC0002A8B3B8B4C8B5D8B0F2D069561F16B81D3
:100ED000102F601708F4162F012FB60180E00E9432
:100EE000A30F892B09F090C08B818F5F811B8B83AF
:100EF000812F90E001979C01442737FD4095542FA6
:100F00008C010F5F1F4F8A899B89AC89BD89820F35
:100F1000931FA41FB51F8A8B9B8BAC8BBD8B102F8F
:100F20000027110F3EC02E813F81488559858A8553
:100F30009B85AC85BD85281739074A075B0790F06C
:100F400060E070E080E090E00E940203882309F4F2
:100F50005BC08A899B89AC89BD89F50184839583AF
:100F6000A683B7836A897B898C899D890E94020345
:100F7000882309F449C02E813F813170C201821B50
:100F8000930B87018E159F0508F48C01205E3F4F5F
:100F90002A0D3B1DA801B601C9010E944B11F501A4
:100FA000378EC00ED11EC801A0E0B0E02E813F8177
:100FB00048855985280F391F4A1F5B1F2E833F83A1
:100FC00048875987F30180819181800F911F918318
:100FD0008083E01AF10AE114F10409F004CF2E81B4
:100FE0003F81488559858A859B85AC85BD8582175B
:100FF0009307A407B50720F42A873B874C875D87B2
:101000008A8180628A8306C08A8180688A8388E0B8
:10101000882E912CC401CDB7DEB7E1E10C94B91153
:10102000A0E0B0E0E6E1F8E00C949E11EC01162F90
:10103000072F7A0139018C809D80F901118210827D
:1010400068817981C4010E94EE025C01009709F079
:10105000F8C08A8187FDF2C080FD04C076E0A72E2B
:10106000B12CEFC02A853B854C855D858E819F81A3
:10107000A885B985281B390B4A0B5B0BC701A0E07B
:10108000B0E0281739074A075B0708F47901812F78
:10109000902F9C016901412C62E0562EC7C02E8121
:1010A0003F8148855985DA01C9019170A070B070FF
:1010B0000097A105B10509F084C08B8181508B8315
:1010C000882349F02A893B894C895D892F5F3F4FEE
:1010D0004F4F5F4F43C0211531054105510519F4AC
:1010E0006E857F8505C0888999890E94FB03BC01B4
:1010F0006230710508F49FC0F401868997896817EA
:10110000790708F098C0798B688B00910A011091DB
:101110000B0162507040F801868997890297681721
:10112000790728F020E030E040E050E014C080E093
:1011300090E0F801258D30E040E050E00E945B1126
:101140009B01AC01F80180899189A289B389280F9C
:10115000391F4A1F5B1FF401858D8B832A8B3B8BC4
:101160004C8B5D8B0F2D069561F16B81102F6017F5
:1011700008F4162F012FB60180E00E94440F892B3E
:1011800009F059C08B818F5F811B8B83812F90E089
:1011900001979C01442737FD4095542F8C010F5F28
:1011A0001F4F8A899B89AC89BD89820F931FA41F19
:1011B000B51F8A8B9B8BAC8BBD8B102F0027110F1B
:1011C0001BC06A897B898C899D890E9402038823C0
:1011D00091F18E819F8191709201281B390B8701BB
:1011E0002E153F0508F489018096880D991DA801E8
:1011F000BC01C6010E944B11C00ED11EC801A0E067
:10120000B0E02E813F8148855985280F391F4A1F3C
:101210005B1F2E833F8348875987F301808191812B
:10122000800F911F91838083E01AF10AE114F10489
:1012300009F035CF06C08A8180688A8348E0A42EF1
:10124000B12CC501CDB7DEB7E0E10C94BA11CF9354
:10125000DF93FB01882319F025E030E01DC0A09149
:101260000A01B0910B0170930B0160930A01109772
:1012700041F080E292E0ED019C0119922150304052
:10128000E1F7309739F080E292E0DF01EC011D9246
:101290002197E9F720E030E0C901DF91CF9108956F
:1012A0000F93CF93DF939B01AC01C0910A01D091C2
:1012B0000B01BE01605E7F4F01E080E00E94440FA1
:1012C000892BC1F4C25EDD4F88819981CE51D24015
:1012D00085559A4A79F443E050E060E071E0CE0130
:1012E0008A5A9F4F0E943E119C0180E0232B19F0E7
:1012F00081E001C082E0DF91CF910F910895ADE1CF
:10130000B0E0E5E8F9E00C949C119D8F8C8F3B01D7
:1013100080900A0190900B01FC011582148203C099
:101320000894611C711CF30180818032C9F38F32F3
:1013300019F40894611C711C8114910409F417C1FB
:10134000F42FFF71FB8F142F1E71F401848D8823FD
:1013500059F080E00E943D0F80FD06C0112309F482
:10136000ABC382FD07C1A8C380E292E0F4019C01F7
:10137000119221503040E1F780E00E94600E80FF22
:1013800003C021E030E08BC3112311F082FDF2C0D5
:1013900060E070E080E090E00E945009813021F030
:1013A000EE24FF2487011EC082EE91E0880E991E74
:1013B000F40180812EE13EEF820E931E882309F412
:1013C000DCC086EE91E0880E991EF401E080F18089
:1013D000028113812AE13EEF820E931EC801B701FC
:1013E0000E945009882309F0C8C0F40183A594A580
:1013F0008050924009F0C1C0F40186A997A9BC01B0
:1014000080E090E0611571058105910569F424E49F
:1014100030E0820E931EF40160817181828193819C
:101420002CEB3FEF820E931EF401758B648B20A989
:10143000268F30E040E050E00E945B115B016C01C0
:10144000F40186A597A5A0E0B0E0E80EF91E0A1FFA
:101450001B1FE086F1860287138785A5858F21A94A
:1014600032A93383228383A994A97C0100E010E090
:10147000E114F1040105110569F480E490E0880E9F
:10148000991EF401E080F1800281138180EC9FEFCE
:10149000880E991EF40186A597A5A0E0B0E0E81A91
:1014A000F90A0A0B1B0BEA18FB080C091D09A4E03A
:1014B00036952795AA95E1F7C901A0E0B0E0E81AB2
:1014C000F90A0A0B1B0B258D30E040E050E0C80103
:1014D000B7010E947A112E5F3F4F4F4F5F4FF401CB
:1014E000378B268B283FFFE03F07F0E04F07F0E007
:1014F0005F0710F461E006C0285F3F4F4040504056
:10150000E0F562E0F4012085318542855385D601FE
:10151000C501820F931FA41FB51F84879587A687D7
:10152000B7878281938174E0969587957A95E1F7E4
:10153000A0E0B0E0820F931FA41FB51F8A0D9B1D72
:10154000AC1DBD1D808B918BA28BB38B648F8FEFF5
:101550009FEF938F828F80910C0190910D010196E6
:1015600090930D0180930C0191838083A5C22AE0A2
:1015700030E095C229E030E092C22BE030E08FC22B
:101580002E010894411C511C92E0292E312C4BE075
:1015900050E060E270E0C2010E94541120E048E097
:1015A00090E038E102C028E04BE0F30111913F01E7
:1015B000112311F01F3249F4222309F4C7C0392343
:1015C0003C87113009F044C0C1C0113208F4BEC0DC
:1015D0001F3709F4BBC01E3241F490FDB7C022236F
:1015E00009F4B4C02930F8F2B1C0123209F4AEC027
:1015F0001A3220F11D3208F4A9C01A33F8F0103461
:1016000008F4A4C090FD1AC01C3709F49FC0812FB4
:101610008B55833008F49AC0865E8A3128F44830AE
:1016200011F4377F01C03F7E812F81568A3130F41B
:101630001052483011F4986001C09061241708F0EE
:1016400085C09E7FF201E20FF11D10832F5FADCFA9
:101650006F89788D898D9A8D0E940203882331F4D9
:1016600090E09C01590128E030E084C02F85388942
:101670002F70307085E0220F331F8A95E1F7F60155
:10168000E20FF31F80A18823E1F0853EA1F000E284
:10169000A02EB12CA20EB31EAC0CBD1CF50183858F
:1016A000082F83FD08C04BE050E0B201C5010E9445
:1016B0003E11009751F0CE010D960E94D40588236B
:1016C00039F6112309F049C04FC0112319F420E065
:1016D00030E050C004FF41C0F501E28CF38CFE8A7B
:1016E000ED8A00910A0110910B01B7016250704020
:1016F000F8018689978902976817790728F020E012
:1017000030E040E050E014C080E090E0F801258D2A
:1017100030E040E050E00E945B119B01AC01F80119
:1017200080899189A289B389280F391F4A1F5B1FBD
:10173000FC8AEB8A2F8B388F498F5A8F388A2F86F5
:1017400026CF20E030E0AA24BB2414C080E090E043
:101750009C01590124E030E00DC080E090E09C0144
:10176000590123E030E006C080E090E09C0159017F
:1017700022E030E0FB8D4F2F50E0CA018C71907059
:10178000892B09F441C12115310509F4D6C0223055
:10179000310509F084C160900A0170900B010B893A
:1017A0001C890115110551F11E8B0D8BB80162507A
:1017B0007040F3018689978902976817790728F0A6
:1017C00020E030E040E050E014C080E090E0F30121
:1017D000258D30E040E050E00E945B119B01AC01A0
:1017E000F30180899189A289B389280F391F4A1F83
:1017F0005B1F2F8B388F498F5A8F09C0F301848567
:101800009585A685B7858F8B988FA98FBA8F188AF3
:101810001F86BDE0EB2EF12CEC0EFD1E6F89788D3E
:10182000898D9A8D0E940203882309F433C1EF85C4
:10183000F889EF70F070A5E0EE0FFF1FAA95E1F7B1
:10184000B0965301AE0EBF1EB097E60DF71D80A1F6
:10185000882309F44CC1853E09F449C1C7010E949F
:10186000D4058823D9F60115110509F410C18D8915
:101870009E890E9479048C01009709F408C1813087
:10188000910509F407C160E070E080E090E00E94FB
:101890000203882309F4FEC0A0900A01B0900B0156
:1018A000B80162507040F5018689978902976817E0
:1018B000790720F0CC24DD24760114C080E090E08C
:1018C000F501258D30E040E050E00E945B116B0196
:1018D0007C01F50180899189A289B389C80ED91E3E
:1018E000EA1EFB1EF301C482D582E682F782E0E2A3
:1018F000AE2EB12CA60CB71C80E092E0F5019C0145
:10190000119221503040E1F7F301158D10C001E034
:10191000A7019601B50180E00E94A30F892B09F071
:10192000B9C00894C11CD11CE11CF11C1150112339
:1019300071F781E0F301878FDAC0F2FF03C027E07F
:1019400030E0ADC0A114B10409F4A1C0F501838554
:10195000817109F09CC043FF42C0C28CD38C138EAE
:10196000128E148E158E168E178E81E0F401878FDD
:101970002480358046805780E0900A01F0900B016A
:1019800086011CC0C8010E94FB033C018130910507
:1019900009F480C060E070E0C8010E946C038823F5
:1019A00009F478C0F701828D938DFFEF8F3F9F0779
:1019B00021F00196F701938F828F83010230110588
:1019C00008F472C0F7018689978908171907D0F2C1
:1019D0006BC00894C108D108F401D18EC08EFB8D74
:1019E000F3FF22C080E2F50183870E94B000F50179
:1019F000668B778B808F918F66877787808B918BB3
:101A000081E0F401878F10C02115310509F047C02E
:101A1000A114B10409F441C0F501838584FD3DC0E2
:101A200041FF02C080FD33C0F40184819581A6810D
:101A3000B781EC8DFD8D868B978BA08FB18FB38E88
:101A4000A28E2B8D2283F501828D938DEC8DFD8DE1
:101A500097878687F501848D958DA68DB78DEC8D42
:101A6000FD8D82879387A487B5871682178210869B
:101A7000118681E0838395828482F4018081918143
:101A8000EC8DFD8D9183808320E030E008C026E05E
:101A900030E005C028E030E002C022E030E0C901BB
:101AA0006D96E2E10C94B811C201B1010E940203EB
:101AB000882309F08ECFEECFC0900A01D0900B01A1
:101AC000F601848595851C8A1B8A1E8A1D8AA0E0E2
:101AD000B0E08F8B988FA98FBA8F188A1F86DA8A09
:101AE000C98AF3018081882309F04ACD2ACE80E299
:101AF000F50111928A95E9F7D501FE0131968BE047
:101B000001900D928150E1F78C85F5018487FB8D62
:101B1000F860FB8F64CFFC018AE080930F019FEF98
:101B20009EBD0DB407FEFDCF8EB58F3F29F4809189
:101B30000F018823A9F722C08E3F01F59FEF9EBDBC
:101B40000DB407FEFDCF8EB580839EBD0DB407FE9C
:101B5000FDCF8EB581836250704011F03296EFCF89
:101B60008FEF8EBD0DB407FEFDCF8EB58FEF8EBD0E
:101B70000DB407FEFDCF8EB581E0089580E0089595
:101B8000FC0182E3809310018FEF8EBD0DB407FE40
:101B9000FDCF8EB59FEF9EBD0DB407FEFDCF8EB578
:101BA0008F3F31F0809110018823A9F790E02EC07B
:101BB0006EBD0DB407FEFDCF6D3F11F491E026C060
:101BC00090E080818EBD0DB407FEFDCF81818EBD7A
:101BD0000DB407FEFDCF915011F03296F2CF8FEF8A
:101BE0008EBD0DB407FEFDCF8FEF8EBD0DB407FE89
:101BF000FDCF8FEF8EBD0DB407FEFDCF8EB590E00B
:101C00008F71853009F091E081E09827892F089540
:101C1000282F82E3809310018FEF8EBD0DB407FE55
:101C2000FDCF8EB59FEF9EBD0DB407FEFDCF8EB5E7
:101C30008F3F31F0809110018823A9F78FEF08952D
:101C40002EBD0DB407FEFDCF872F9927AA27BB27EE
:101C50008EBD0DB407FEFDCFCB01AA27BB278EBDDD
:101C60000DB407FEFDCFBB27A72F962F852F8EBD66
:101C70000DB407FEFDCF4EBD0DB407FEFDCF2034E1
:101C800011F485E905C0283411F487E801C080E02B
:101C90008EBD0DB407FEFDCF2C3431F48FEF8EBD19
:101CA0000DB407FEFDCF8EB59AE02FEF2EBD0DB41B
:101CB00007FEFDCF8EB587FF02C09150B9F708959A
:101CC000A4E0B0E0E6E6FEE00C94A811882311F051
:101CD00081E0CFC08091040181FDC9C08AE09FEFFF
:101CE0009EBD0DB407FEFDCF2EB58150C9F72A98D1
:101CF00040E050E060E070E080E40E94080E813037
:101D000009F0A0C084E680930F014AEA51E060E048
:101D100070E088E40E94080E813009F054C07E0112
:101D20000894E11CF11C87019FEF9E012B5F3F4F40
:101D30009EBD0DB407FEFDCF8EB5F80181938F01D6
:101D4000E217F307A9F78B81813009F07BC08C8102
:101D50008A3A09F077C040E050E060E070E087E741
:101D60000E94080E823048F440E050E060E070E4E9
:101D700089E60E94080E882321F080910F018823B4
:101D800051F780910F01882309F45CC040E050E0D6
:101D900060E070E08AE70E94080E882309F052C0D4
:101DA0009FEF9EBD0DB407FEFDCF8EB5F701819369
:101DB0007F01E017F107A9F7898186FD02C012E0D3
:101DC00042C016E040C040E050E060E070E087E7CD
:101DD0000E94080E823058F440E050E060E070E06D
:101DE00089E60E94080E823010F412E001C011E072
:101DF000123079F440E050E060E070E087E70E9444
:101E0000080E823078F440E050E060E070E089E64F
:101E100005C040E050E060E070E081E40E94080E00
:101E2000882321F080910F01882311F780910F0101
:101E3000882341F040E052E060E070E080E50E94DD
:101E4000080E811110E0109311012A9A8FEF8EBDB8
:101E50000DB407FEFDCF8EB5112321F08091040152
:101E60008E7F03C080910401816080930401809182
:101E700004012496E6E00C94C411882311F081E05B
:101E800008958091040108950F93CF93DF93EB01A0
:101E9000882309F051C0002309F44EC08091040149
:101EA00080FF03C023E030E049C08091110182FD32
:101EB00007C069E0220F331F441F551F6A95D1F7F1
:101EC0002A98013089F4BA01A90181E50E94080E1F
:101ED000882321F560E072E0CE010E948B0D00E0C6
:101EE0008823E1F401E01AC0BA01A90182E50E9449
:101EF000080E882399F460E072E0CE010E948B0DF9
:101F0000882329F0015019F0C050DE4FF4CF40E093
:101F100050E060E070E08CE40E94080E2A9A8FEF97
:101F20008EBD0DB407FEFDCF8EB520E030E000235E
:101F300029F021E030E002C024E030E0C901DF9167
:101F4000CF910F910895CF92DF92EF92FF920F936E
:101F5000CF93DF93EB0169017A01882309F064C014
:101F6000002309F461C08091040180FF03C023E0D5
:101F700030E05CC08091040182FF03C022E030E0C9
:101F800055C08091110182FD07C079E0CC0CDD1CA9
:101F9000EE1CFF1C7A95D1F72A98013069F4B7013D
:101FA000A60188E50E94080E882381F56EEFCE0118
:101FB0000E94C00D00E027C081FF0EC040E050E04D
:101FC00060E070E087E70E94080E402F50E060E07C
:101FD00070E087E50E94080EB701A60189E50E941E
:101FE000080E882399F46CEFCE010E94C00D88235F
:101FF00029F0015019F0C050DE4FF5CF6DEF80E0B1
:1020000090E00E94C00D882309F401E02A9A8FEF26
:102010008EBD0DB407FEFDCF8EB520E030E000236D
:1020200029F021E030E002C024E030E0C901DF9176
:10203000CF910F91FF90EF90DF90CF900895A0E1A6
:10204000B0E0E5E2F0E10C94AA118A01882319F0CE
:1020500024E030E0E7C02A98633009F47FC06430A0
:1020600028F4613079F0623051F472C06B3009F4B9
:1020700096C06C3009F4AAC06A3009F486C024E026
:1020800030E0C6C040E050E060E070E089E40E94CB
:10209000080E882309F0B7C060E170E0CE01019618
:1020A0000E948B0D882309F4AEC0898182958695A4
:1020B000869583707A8549858130B1F4872F90E0C9
:1020C0000196342F20E0820F931FA0E0B0E02AE0B9
:1020D000880F991FAA1FBB1F2A95D1F7F80180838B
:1020E0009183A283B38392C04295469546954370EF
:1020F000288530E0220F331F220F331F240F311D9C
:102100002F5F3F4F8F8190E083709070982F8827CA
:10211000990F990F280F391F40E050E08E818F7082
:102120006B85661F6627661F860F8E5F7370770F3D
:10213000870F90E0099704C0220F331F441F551FDB
:102140008A95D2F7F80120833183428353835EC09E
:1021500080E092E0FA019183808358C082E380930B
:1021600010018FEF8EBD0DB407FEFDCF8EB59FEF32
:102170009EBD0DB407FEFDCF8EB58F3F09F446C05E
:10218000809110018823A1F73EC08091040180FD59
:1021900047C040E050E060E070E089E409C0809111
:1021A000040180FD3DC040E050E060E070E08AE462
:1021B0000E94080E882339F560E170E0C8010E9492
:1021C0008B0D20E030E0882319F51DC080910401BB
:1021D00080FD26C040E050E060E070E08AE70E94A9
:1021E000080E882381F4F8019FEF98012D5F3F4F7F
:1021F0009EBD0DB407FEFDCF8EB58083E217F307B9
:1022000029F03196F5CF21E030E002C020E030E047
:102210002A9A8FEF8EBD0DB407FEFDCF8EB502C09A
:1022200023E030E0C9016096E4E00C94C61180918F
:102230000F01882319F0815080930F0180911001C4
:10224000882319F081508093100190910E0183B181
:10225000817080930E01981749F48091040190FFDA
:1022600002C0836001C08D7F809304010895FB014B
:10227000DC0105900D920020E1F70895FB01DC01DF
:1022800004C08D910190801921F441505040C8F74D
:10229000881B990B0895FB01DC0102C001900D928F
:1022A00041505040D8F70895DC0101C06D93415072
:1022B0005040E0F70895629FD001739FF001829F24
:1022C000E00DF11D649FE00DF11D929FF00D839FC5
:1022D000F00D749FF00D659FF00D9927729FB00D62
:1022E000E11DF91F639FB00DE11DF91FBD01CF0175
:1022F00011240895A1E21A2EAA1BBB1BFD010DC0DB
:10230000AA1FBB1FEE1FFF1FA217B307E407F507A5
:1023100020F0A21BB30BE40BF50B661F771F881F81
:10232000991F1A9469F760957095809590959B0117
:10233000AC01BD01CF0108952F923F924F925F9261
:102340006F927F928F929F92AF92BF92CF92DF92C5
:10235000EF92FF920F931F93CF93DF93CDB7DEB72A
:10236000CA1BDB0B0FB6F894DEBF0FBECDBF0994BE
:102370002A88398848885F846E847D848C849B8415
:10238000AA84B984C884DF80EE80FD800C811B8123
:10239000AA81B981CE0FD11D0FB6F894DEBF0FBE52
:0A23A000CDBFED010895F894FFCFC2
:0623AA0046415400010051
:00000001FF
